:100000000C947A000C9497000C9497000C94970031
:100010000C9497000C9497000C9497000C94970004
:100020000C9497000C9497000C9497000C949700F4
:100030000C9497000C9497000C9497000C949700E4
:100040000C9497000C9437240C9497000C94970010
:100050000C9497000C9497000C9497000C949700C4
:100060000C9497000C946E090C9497000C94AC09B6
:100070000C9497000C9497000C9497000C949700A4
:100080000C9497000C9497000C9497000C94970094
:100090000C9497000C9497000C9497000C94970084
:1000A0000C9497000C9497000C9497000C94970074
:1000B0000C9497000C9497000C9497000C94970064
:1000C0000C9497000C9497000C9497000C94970054
:1000D0000C9497000C9497000C9497000C94970044
:1000E0000C949700000000000000000000000000D9
:1000F0000000000011241FBECFEFD1E2DEBFCDBF54
:1001000017E0A0E0B2E0EEE8FBE400E00BBF02C0C5
:1001100007900D92A03BB107D9F712E1A0EBB7E031
:1001200001C01D92AA32B107E1F70C9499000C941A
:100130000000EF92FF920F93CF93DF93CDB7DEB71E
:10014000E1E0F1E088E38083EAE0F1E088E38083A6
:10015000EDE2F0E08AEF8083E7E0F1E08FE080837A
:10016000EEE2F0E01082E2E0F1E01082E8E0F1E09F
:100170001082EBE0F1E0108201E020E048E060E076
:1001800070E081EE97E40E94EF0961E085E00E9453
:10019000C115909329128093281261E085E00E9496
:1001A000C115909327128093261280E090E00E9460
:1001B000F80B87E092E0EAE0F1E0EE24FF2401E0B2
:1001C00020E030E04CE251E0BC01CF010E942E0E55
:1001D0008FE092E0EDE9F1E0EE24FF2401E020E081
:1001E00030E048E552E0BC01CF010E942E0E84E1D0
:1001F00092E0EEE2F1E0EE24FF2402E020E030E0C5
:1002000048E552E0BC01CF010E942E0E0E94691009
:100210000000FECFCF93DF93CDB7DEB722970FB6A6
:10022000F894DEBF0FBECDBF9A838983A8E0B1E00A
:10023000E8E0F1E0808181608C9384EF91E00E949E
:100240000710A8E0B1E0E8E0F1E090818EEF8923AB
:100250008C9384EF91E00E940710E8CFCF93DF9357
:10026000CDB7DEB727970FB6F894DEBF0FBECDBF70
:100270009F838E830E94980B8D838D8183330CF432
:1002800054C08EE192E00E94D30888EE93E00E9471
:1002900007100FB6F8940F92EEE2F0E080818C83A5
:1002A000E2E0F1E080818B83EBE0F1E080818A8302
:1002B000E8E0F1E080818983AEE2B0E0EEE2F0E0D8
:1002C000908187EC89238C93A2E0B1E0E2E0F1E039
:1002D000908187EC89238C93ABE0B1E0EBE0F1E017
:1002E000908187EC89238C93E8E0F1E088E08083BB
:1002F00003C00E94980B8D838D818E32D4F7E8E085
:10030000F1E089818083EEE2F0E08C818083E2E09D
:10031000F1E08B818083EBE0F1E08A81808387E7E5
:1003200092E00E94D3080F900FBE88EE93E00E94E7
:1003300007100E94980B8D83A0CFCF93DF93CDB78A
:10034000DEB7A7970FB6F894DEBF0FBECDBF9DA353
:100350008CA383E892E00E94D30883E892E00E9495
:10036000D3088CE992E00E94D3080E94030400C0E5
:100370008DE00E9415098AE00E9415098EE30E9413
:1003800015091D82CE0106960E944C098E810E949D
:10039000150917C08D818F5F8D838D8199279C01F1
:1003A000CE010696820F931F0E944C098D81282F43
:1003B0003327CE010696FC01E20FF31F80810E94D5
:1003C00015098D81282F3327CE010696FC01E20FF7
:1003D000F31F80818D3019F08D818930D8F28D81A5
:1003E000282F3327CE010696FC01E20FF31F10825F
:1003F0008AE00E9415098E81282F33273FA32EA360
:100400004EA15FA14435510509F4B4C18EA19FA14D
:1004100085359105ECF52EA13FA12333310509F473
:10042000EAC14EA15FA1443351059CF48EA19FA166
:100430008133910509F4D9C12EA13FA122333105A1
:100440000CF0D6C14EA15FA14332510509F4B6C0EC
:10045000D5C18EA19FA18534910509F4E1C02EA1DB
:100460003FA1263431056CF44EA15FA14F335105F5
:1004700009F448C08EA19FA18434910509F40FC1ED
:10048000BDC12EA13FA12235310509F44DC1B6C130
:100490004EA15FA14D36510509F44CC08EA19FA11C
:1004A0008E36910594F42EA13FA12536310509F42D
:1004B000B7C04EA15FA14736510551F18EA19FA152
:1004C0008436910509F4EBC099C12EA13FA12237D2
:1004D000310509F429C14EA15FA14337510534F418
:1004E0008EA19FA18037910581F088C12EA13FA1E7
:1004F0002437310509F43EC14EA15FA147375105AC
:10050000B9F17CC10E94030433CF0E943A0430CF7A
:100510001D8205C00E9485058D818F5F8D838D8131
:10052000282F33278091050290910602281739075A
:1005300088F31ECFCE01069601960E943A24AA2780
:1005400097FDA095BA2F89839A83AB83BC83898159
:100550009A81AB81BC818093B0079093B107A0933F
:10056000B207B093B3078FEC92E00E94D30800CF9C
:10057000CE01069601960E943A24AA2797FDA095DF
:10058000BA2F89839A83AB83BC8389819A81AB819B
:10059000BC8185309105A105B1052CF483ED92E075
:1005A0000E94D308E5CE89819A81909301028093BD
:1005B00000028FEC92E00E94D308DACECE010696BC
:1005C00001960E943A24AA2797FDA095BA2F898305
:1005D0009A83AB83BC8389819A81AB81BC818F3F35
:1005E0009105A105B10531F02CF08EEF92E00E944B
:1005F000D308BECE89819A81AB81BC8118161906B9
:100600001A061B062CF086E293E00E94D308B0CEB7
:100610008981809304028FEC92E00E94D308A8CED7
:10062000CE01069601960E943A24AA2797FDA0952E
:10063000BA2F89839A83AB83BC8389819A81AB81EA
:10064000BC818A309105A105B1054CF489819A815C
:10065000AB81BC81181619061A061B062CF086E51C
:1006600093E00E94D30884CE89819A8101979C01EE
:1006700081E090E002C0880F991F2A95E2F79C0163
:100680008091020290910302822B932B909303029C
:10069000809302028FEC92E00E94D30869CECE01D3
:1006A000069601960E943A24AA2797FDA095BA2F94
:1006B00089839A83AB83BC8389819A81AB81BC8116
:1006C0008A309105A105B1054CF489819A81AB81ED
:1006D000BC81181619061A061B062CF086E593E055
:1006E0000E94D30845CE89819A8101979C0181E0BF
:1006F00090E0AC0102C0440F551F2A95E2F79A0121
:100700008FEF91E0821B930B9C01809102029091EC
:1007100003028223932390930302809302028FECBF
:1007200092E00E94D30824CECE01069601960E9444
:100730003A24AA2797FDA095BA2F89839A83AB8381
:10074000BC8389819A81AB81BC81181619061A066F
:100750001B062CF080E993E00E94D30809CE898122
:100760009A8190930602809305028FEC92E00E949A
:10077000D308FECD8DEB93E00E94D3080E94980B26
:10078000282F332727FD3095CE0140964AE050E0D0
:10079000BC01C9010E948624CE0140960E94D30864
:1007A00087EA0E9415098FED93E00E94D30884EE3A
:1007B00093E00E94D3080E94550B282F332727FD72
:1007C0003095CE0140964AE050E0BC01C9010E943C
:1007D0008624CE0140960E94D30887EA0E9415091C
:1007E0008FED93E00E94D308C3CD0E94B207C0CD25
:1007F0000E941108BDCD0E946308BACD89E094E043
:100800000E94D308B5CDCF93DF93CDB7DEB784E395
:1008100094E00E94D30887E494E00E94D30888E51E
:1008200094E00E94D30881E794E00E94D3088AE80C
:1008300094E00E94D30888EB94E00E94D30881E002
:1008400095E00E94D30882E495E00E94D30884E8F2
:1008500095E00E94D30886EA95E00E94D30889ECCF
:1008600095E00E94D3088BEE95E00E94D308DF91BB
:10087000CF910895CF93DF93CDB7DEB764970FB6CE
:10088000F894DEBF0FBECDBF85E096E00E94D3088E
:1008900081E296E00E94D3088091B0079091B10761
:1008A000A091B207B091B3070097A105B10529F453
:1008B0008BE396E00E94D3081DC087E596E00E9476
:1008C000D3088091B0079091B107A091B207B09181
:1008D000B3079C014AE050E0CE010196BC01C9017A
:1008E0000E948624CE0101960E94D3088FE696E0EE
:1008F0000E94D30885E796E00E94D3088091000209
:10090000909101029C014AE050E0CE010196BC01A9
:10091000C9010E948624CE0101960E94D3088FE669
:1009200096E00E94D30883E996E00E94D308809164
:100930000402282F33274AE050E0CE010196BC0183
:10094000C9010E948624CE0101960E94D30887EA3D
:1009500096E00E94D3088BEA96E00E94D30880912B
:100960000502909106029C014AE050E0CE010196FA
:10097000BC01C9010E948624CE0101960E94D308C1
:100980008EEB96E00E94D3088BEC96E00E94D30891
:10099000809102029091030281709070882321F06F
:1009A0008FED96E00E94D30880910202909103029D
:1009B000867090708630910529F483EF96E00E944E
:1009C000D30818C080910202909103028270907047
:1009D000009721F08DE097E00E94D30880910202F9
:1009E0009091030284709070009721F087E297E065
:1009F0000E94D30880910202909103028870907047
:100A0000009721F081E497E00E94D30880910202D0
:100A10009091030280719070009721F081E597E03A
:100A20000E94D3088091020290910302807290701C
:100A3000009721F082E697E00E94D308809102029D
:100A40009091030280749070009721F083E797E003
:100A50000E94D308809102029091030280789070E6
:100A6000009721F082E897E00E94D308809102026B
:100A70009091030280709170009721F086E997E0D1
:100A80000E94D3088DEB93E00E94D3080E94980B3C
:100A9000282F332727FD30954AE050E0CE010196FC
:100AA000BC01C9010E948624CE0101960E94D30890
:100AB00087EA0E9415098FED93E00E94D30884EE27
:100AC00093E00E94D3080E94550B282F332727FD5F
:100AD00030954AE050E0CE010196BC01C9010E9468
:100AE0008624CE0101960E94D30887EA0E94150948
:100AF0008FED93E00E94D30864960FB6F894DEBFA2
:100B00000FBECDBFDF91CF910895CF93DF93CDB7C7
:100B1000DEB722970FB6F894DEBF0FBECDBF1A82A4
:100B2000A8E0B1E0E8E0F1E0808184608C931A8273
:100B300083C0198278C08A81282F332781E090E012
:100B400002C0880F991F2A95E2F79C01809102024A
:100B500090910302A901482359238A81282F332722
:100B600081E090E0022E02C0880F991F0A94E2F7FC
:100B70004817590709F054C080910202909103026E
:100B8000867090708630910521F48A81823009F454
:100B900047C08091B0079091B107A091B207B09182
:100BA000B3070097A105B10589F48A810E944E061A
:100BB0000E94310680910002909101020E9407106C
:100BC0000E943F068A810E94E80626C00E943106E4
:100BD00089E190E00E9407100E943F0689E190E0C1
:100BE0000E9407108091B0079091B107A091B207C1
:100BF000B091B3070E9407108A810E944E060E949E
:100C0000310680910002909101020E9407100E941B
:100C10003F068A810E94E8068AE090E00E94071061
:100C200089818F5F8983909104028981891708F4F3
:100C300082CF8A818F5F8A838A81893008F479CF55
:100C4000A8E0B1E0E8E0F1E090818BEF89238C939C
:100C500022960FB6F894DEBF0FBECDBFDF91CF91C5
:100C60000895CF93DF93CDB7DEB7A4E3B0E0E4E31C
:100C7000F0E0808183608C93DF91CF910895CF93D2
:100C8000DF93CDB7DEB7A4E3B0E0E4E3F0E090811A
:100C90008CEF89238C93DF91CF910895CF93DF93CD
:100CA000CDB7DEB723970FB6F894DEBF0FBECDBF2A
:100CB00089838981282F33273B832A838A819B81DB
:100CC0008430910509F455C02A813B8125303105D6
:100CD000D4F48A819B818130910579F12A813B810D
:100CE000223031052CF48A819B81009709F167C07D
:100CF0002A813B812230310591F18A819B818330A9
:100D0000910591F15CC02A813B8126303105D9F1F2
:100D10008A819B81863091058CF12A813B81273025
:100D20003105B1F18A819B8188309105E9F147C095
:100D3000EEE2F0E088E0808342C080910202909170
:100D4000030284709070009729F0EEE2F0E080E3F7
:100D5000808335C0EEE2F0E080E1808330C0EEE2D7
:100D6000F0E080E280832BC0E2E0F1E088E0808365
:100D700026C0E2E0F1E080E1808321C0E2E0F1E022
:100D800080E280831CC0EBE0F1E088E0808317C044
:100D9000EBE0F1E080E18083A8E0B1E0E8E0F1E0A1
:100DA000808182608C930BC0EBE0F1E080E2808375
:100DB000A8E0B1E0E8E0F1E0808182608C932396C6
:100DC0000FB6F894DEBF0FBECDBFDF91CF9108956F
:100DD000CF93DF93CDB7DEB723970FB6F894DEBF7E
:100DE0000FBECDBF89838981282F33273B832A8378
:100DF0008A819B818430910509F46FC02A813B81EF
:100E000025303105E4F48A819B8181309105C9F157
:100E10002A813B81223031052CF48A819B81009705
:100E200039F197C02A813B812230310509F443C052
:100E30008A819B818330910509F446C08AC02A814A
:100E40003B812630310509F45AC08A819B81863066
:100E500091050CF44BC02A813B812730310509F400
:100E600057C08A819B818830910509F462C071C0A6
:100E7000AEE2B0E0EEE2F0E0908187EF89238C9360
:100E800068C0809102029091030284709070009774
:100E900049F0AEE2B0E0EEE2F0E090818FEC892321
:100EA0008C9357C0AEE2B0E0EEE2F0E090818FEEBE
:100EB00089238C934EC0AEE2B0E0EEE2F0E0908188
:100EC0008FED89238C9345C0A2E0B1E0E2E0F1E030
:100ED000908187EF89238C933CC0A2E0B1E0E2E0EF
:100EE000F1E090818FEE89238C9333C0A2E0B1E0D2
:100EF000E2E0F1E090818FED89238C932AC0ABE092
:100F0000B1E0EBE0F1E0908187EF89238C9321C081
:100F1000ABE0B1E0EBE0F1E090818FEE89238C93C0
:100F2000A8E0B1E0E8E0F1E090818DEF89238C93B7
:100F300010C0ABE0B1E0EBE0F1E090818FED8923F0
:100F40008C93A8E0B1E0E8E0F1E090818DEF892397
:100F50008C9323960FB6F894DEBF0FBECDBFDF9102
:100F6000CF910895CF93DF93CDB7DEB724970FB617
:100F7000F894DEBF0FBECDBF1C821B8243C01A8215
:100F8000198213C081E00E944E0688E290E00E9420
:100F9000071081E00E94E8068EE190E00E940710B1
:100FA00089819A8101969A83898389819A8188307F
:100FB000910544F38EE190E00E9407101A82198295
:100FC00013C086E00E944E0688E290E00E9407105F
:100FD00086E00E94E8068EE190E00E940710898179
:100FE0009A8101969A83898389819A8188309105B3
:100FF00044F38EE190E00E9407108B819C81019662
:101000009C838B838B819C818A3091050CF4B7CFB4
:1010100024960FB6F894DEBF0FBECDBFDF91CF91FF
:101020000895CF93DF93CDB7DEB724970FB6F8942A
:10103000DEBF0FBECDBF1C821B822DC081E00E948F
:101040004E0682E090E00E94071081E00E94E806D0
:1010500083E00E944E0683E090E00E94071083E048
:101060000E94E80684E00E944E0682E090E00E9422
:10107000071084E00E94E80686E00E944E0682E0A7
:1010800090E00E94071086E00E94E8068B819C8118
:1010900001969C838B838B819C8121E0843F920706
:1010A0006CF282E00E94E80684E00E94E80686E096
:1010B0000E94E80624960FB6F894DEBF0FBECDBF9F
:1010C000DF91CF910895CF93DF93CDB7DEB781E065
:1010D0000E944E0688E592E00E94071081E00E947F
:1010E000E80683E00E944E0688E592E00E94071021
:1010F00083E00E94E80684E00E944E0688E592E0C4
:101100000E94071084E00E94E80686E00E944E06D6
:1011100088E592E00E94071086E00E94E80680E9D8
:1011200091E00E94071082E00E944E0686E00E9435
:101130004E0688EE93E00E94071082E00E94E806C7
:1011400086E00E94E80682E00E944E0684E00E944B
:101150004E0688EE93E00E94071082E00E94E806A7
:1011600084E00E94E806E2E0F1E088E2808388EE15
:1011700093E00E940710E2E0F1E0108281E00E941B
:10118000E80682E00E94E80683E00E94E80684E028
:101190000E94E80685E00E94E80686E00E94E806D4
:1011A000DF91CF910895CF93DF93CDB7DEB724972A
:1011B0000FB6F894DEBF0FBECDBF9C838B831A821F
:1011C0001982A8E0B1E0E8E0F1E0808188608C93CA
:1011D00010C089819A819C018B819C81F901E80F63
:1011E000F91F80810E94150989819A8101969A834D
:1011F000898389819A819C018B819C81F901E80F07
:10120000F91F8081882329F7A8E0B1E0E8E0F1E048
:10121000908187EF89238C9324960FB6F894DEBFD4
:101220000FBECDBFDF91CF910895CF93DF93CDB7A0
:10123000DEB721970FB6F894DEBF0FBECDBF89830E
:1012400080912612909127120E942419882369F414
:10125000E0ECF0E08081992780729070009729F08F
:10126000E6ECF0E0898180830EC080912612909197
:1012700027124FEF50E09E012F5F3F4FB9010E94B0
:101280006616813091F721960FB6F894DEBF0FBE37
:10129000CDBFDF91CF910895CF93DF93CDB7DEB768
:1012A00022970FB6F894DEBF0FBECDBF9A83898315
:1012B000809128129091291229813A814FEF50E0B4
:1012C000B9010E94C717813099F722960FB6F8949A
:1012D000DEBF0FBECDBFDF91CF9108951F920F9259
:1012E0000FB60F9211242F933F934F935F936F93F9
:1012F0007F938F939F93AF93BF93EF93FF93CF937E
:10130000DF93CDB7DEB72197DEBFCDBFE6ECF0E0CF
:1013100080818983209128123091291240E0CE01EA
:101320000196BC01C9010E9443172196F894DEBFC3
:10133000CDBFDF91CF91FF91EF91BF91AF919F9181
:101340008F917F916F915F914F913F912F910F906E
:101350000FBE0F901F9018951F920F920FB60F920D
:1013600011242F933F934F935F936F937F938F93AA
:101370009F93AF93BF93EF93FF93CF93DF93CDB73B
:10138000DEB72297DEBFCDBF1A82CE010296209132
:10139000261230912712AC01CE010196BC01C90181
:1013A0000E94A118813021F4E6ECF0E0898180836D
:1013B0002296F894DEBFCDBFDF91CF91FF91EF91E0
:1013C000BF91AF919F918F917F916F915F914F915D
:1013D0003F912F910F900FBE0F901F9018950F9374
:1013E000CF93DF93CDB7DEB72D970FB6F894DEBF5E
:1013F0000FBECDBF6B837C838D839E834F832887F5
:10140000098720E030E040E85FE36B817C818D81DB
:101410009E810E94BF24DC01CB019C01AD0160E0F4
:1014200074E284E799E40E940225DC01CB01BC014F
:10143000CD010E944825DC01CB019A838983E5EC2C
:10144000F0E089819A81892F99278F708083E4EC5D
:10145000F0E089818083A1ECB0E0E1ECF0E08081F4
:1014600088618C93A1ECB0E0E1ECF0E080818068D1
:101470008C93A1ECB0E0E1ECF0E0808180648C938F
:10148000A2ECB0E0E2ECF0E090818FE389238C9352
:101490008F81282F332727FD30953D872C878C851A
:1014A0009D858730910591F12C853D85283031054A
:1014B0005CF48C859D858530910589F02C853D8572
:1014C00026303105A1F048C08C859D858830910576
:1014D00061F12C853D8529303105B1F13DC0A2EC8B
:1014E000B0E0E2ECF0E08081817F8C9343C0A2EC1D
:1014F000B0E0E2ECF0E08081897F8C93A2ECB0E078
:10150000E2ECF0E0808182608C9334C0A2ECB0E029
:10151000E2ECF0E08081817F8C93A2ECB0E0E2EC21
:10152000F0E0808184608C9325C0A2ECB0E0E2EC16
:10153000F0E080818B7F8C93A2ECB0E0E2ECF0E0F5
:10154000808186608C9316C0A2ECB0E0E2ECF0E003
:1015500080818E608C930EC0A2ECB0E0E2ECF0E0F3
:1015600080818B7F8C93A2ECB0E0E2ECF0E0808194
:1015700086608C93A2ECB0E0E2ECF0E08081282F52
:101580008985992787FD90950197880F991F880F66
:10159000991F880F991F822B8C93A2ECB0E0E2EC8C
:1015A000F0E08081282F8985992787FD9095019704
:1015B000880F991F880F991F880F991F876F8223A3
:1015C0008C938885282F332727FD30953B872A87E2
:1015D0008A859B858130910591F02A853B85223053
:1015E0003105A9F08A859B85009709F01FC0A2EC00
:1015F000B0E0E2ECF0E080818F7C8C931EC0A2EC26
:10160000B0E0E2ECF0E0808180638C9316C0A2EC45
:10161000B0E0E2ECF0E080818F7E8C93A2ECB0E051
:10162000E2ECF0E0808180628C9307C0A2ECB0E035
:10163000E2ECF0E080818F7C8C932D960FB6F894CD
:10164000DEBF0FBECDBFDF91CF910F910895CF9335
:10165000DF93CDB7DEB70E94771EDF91CF9108955B
:10166000CF93DF93CDB7DEB721970FB6F894DEBFE7
:101670000FBECDBF8983ECEBF0E090E88981892B28
:101680008083ECEBF0E080818823DCF7E9EBF0E08D
:101690008081992787FD909521960FB6F894DEBF3B
:1016A0000FBECDBFDF91CF910895CF93DF93CDB71C
:1016B000DEB722970FB6F894DEBF0FBECDBF84EA27
:1016C0000E94300BEBEBF0E080E9808384E80E941D
:1016D000300BEBEBF0E0108284E80E94300B84EAE0
:1016E0000E94300BEBEBF0E081E9808384E80E94FC
:1016F000300B84EC0E94300BEBEBF0E080818A83AE
:1017000084E80E94300BEBEBF0E080818983ECEB06
:10171000F0E084E980838A81992787FD909522965D
:101720000FB6F894DEBF0FBECDBFDF91CF91089505
:10173000CF93DF93CDB7DEB722970FB6F894DEBF15
:101740000FBECDBF84EA0E94300BEBEBF0E082E9E4
:10175000808384E80E94300BEBEBF0E0108284E899
:101760000E94300B84EA0E94300BEBEBF0E083E93F
:10177000808384E80E94300B84EC0E94300BEBEBFA
:10178000F0E080818A8384E80E94300BEBEBF0E08C
:1017900080818983ECEBF0E084E980838A8199275A
:1017A00087FD909522960FB6F894DEBF0FBECDBF91
:1017B000DF91CF910895CF93DF93CDB7DEB7239715
:1017C0000FB6F894DEBF0FBECDBF8B83CE0101965E
:1017D00042E0BC0188E40E948D0D89819A812396A4
:1017E0000FB6F894DEBF0FBECDBFDF91CF91089545
:1017F000CF93DF93CDB7DEB722970FB6F894DEBF55
:101800000FBECDBF9A838983EAE2F0E083E0808354
:10181000ABE2B0E0EBE2F0E0808183608C938AE0A1
:101820000E94F40C22960FB6F894DEBF0FBECDBF17
:10183000DF91CF910895CF93DF93CDB7DEB7229795
:101840000FB6F894DEBF0FBECDBFECEBF0E084E93D
:1018500080838091B5078093B4078091B407882373
:1018600041F0ECEBF0E08081992780719070009757
:10187000A1F7ECEBF0E080819927807190700097E0
:1018800029F081E090E09A83898302C01A8219824C
:1018900089819A8122960FB6F894DEBF0FBECDBF24
:1018A000DF91CF910895CF93DF93CDB7DEB7249723
:1018B0000FB6F894DEBF0FBECDBF89836A83ECEB11
:1018C000F0E084EA80838091B5078093B40780912B
:1018D000B407882329F0ECEBF0E080818823BCF783
:1018E000ECEBF0E084E08083ECEBF0E08081882397
:1018F0002CF082E090E09C838B836BC0E9EBF0E0FE
:1019000080819927887F90708830910529F083E045
:1019100090E09C838B835DC0EBEBF0E0898199279D
:10192000880F991F982F8A818170892B8083ECEB17
:10193000F0E084E880838091B5078093B4078091BC
:10194000B407882329F0ECEBF0E080818823BCF712
:10195000ECEBF0E0808188232CF084E090E09C8325
:101960008B8337C08A818130C9F4E9EBF0E0808154
:101970009927887F90708034910549F1E9EBF0E078
:1019800080819927887F90708834910511F40E9496
:101990001B0C85E090E09C838B831BC0E9EBF0E09F
:1019A00080819927887F90708831910581F0E9EBDB
:1019B000F0E080819927887F90708032910511F442
:1019C0000E941B0C86E090E09C838B8302C01C82EB
:1019D0001B828B819C8124960FB6F894DEBF0FBECC
:1019E000CDBFDF91CF910895CF93DF93CDB7DEB711
:1019F00021970FB6F894DEBF0FBECDBF89838981D2
:101A00008093B507E9EBF0E01082E8EBF0E088E4C2
:101A1000808321960FB6F894DEBF0FBECDBFDF9155
:101A2000CF910895CF93DF93CDB7DEB727970FB649
:101A3000F894DEBF0FBECDBF8A837C836B834D835A
:101A400060E08A810E94530C89838981882331F068
:101A50008981282F33273F832E8354C0ABEBB0E01E
:101A6000EB81FC8180818C938B819C8101969C838E
:101A70008B83ECEBF0E084E880838091B507809362
:101A8000B4078091B407882329F0ECEBF0E0808163
:101A90008823BCF7ECEBF0E0808188232CF087E012
:101AA00090E09F838E832EC0E9EBF0E08081992740
:101AB000887F90708832910581F0E9EBF0E08081B9
:101AC0009927887F90708033910511F40E941B0C38
:101AD00028E030E03F832E8315C08D8181508D83B7
:101AE0008D81882309F0BACF0E941B0C89838981DC
:101AF000882331F08981282F33273F832E8302C02A
:101B00001F821E828E819F8127960FB6F894DEBFBA
:101B10000FBECDBFDF91CF910895CF93DF93CDB7A7
:101B2000DEB72E970FB6F894DEBF0FBECDBF8A8307
:101B30007C836B834D8361E08A810E94530C89838F
:101B40008981882331F08981282F33273E872D878B
:101B50006AC08CEB90E09C878B878D81813019F077
:101B600094EC9A8702C0E4E8EA872A85EB85FC8535
:101B700020838091B5078093B4078091B4078823B0
:101B800029F0ECEBF0E080818823BCF7ECEBF0E08F
:101B9000808188232CF089E090E09E878D8743C068
:101BA000E9EBF0E080819927FC01E87FF070F9878C
:101BB000E8878D81813029F020E530E03F832E8356
:101BC00004C088E590E09F838E83E885F9852E81A7
:101BD0003F81E217F30739F00E941B0C8AE090E086
:101BE0009E878D8720C0EBEBF0E08081EB81FC814C
:101BF00080838B819C8101969C838B838D81815016
:101C00008D838D81882309F0A4CF0E941B0C8983CA
:101C10008981882331F08981E82FFF27FE87ED87AE
:101C200002C01E861D868D859E852E960FB6F89461
:101C3000DEBF0FBECDBFDF91CF910895CF93DF936D
:101C4000CDB7DEB78091B407882329F08091B4071F
:101C500081508093B407DF91CF910895EF92FF9266
:101C60000F93CF93DF93CDB7DEB760970FB6F8949D
:101C7000DEBF0FBECDBF9F838E83798768875B876A
:101C80004A873D872C870E87F88AEF868A859B8551
:101C90000E9460159C838B838B819C81009709F443
:101CA0008DC0888599856A857B85EB81FC812E8531
:101CB000AC01CF010E946D14EB81FC812789308D2E
:101CC000EB81FC8182A193A1820F931F01979A83DC
:101CD00089838C859D852E813F81E981FA81AC01C4
:101CE000B901CF010E945421EB81FC819183808353
:101CF0000FB6F8940F928091B9078F5F8093B90760
:101D00008091B907813049F48B819C819093B7070A
:101D10008093B6070E94C41412C08091BE07882326
:101D200071F4E091B607F091B70796898E8589170F
:101D300030F08B819C819093B7078093B607EB813D
:101D4000FC8196898091BC07891728F4EB81FC817E
:101D500086898093BC078091C307EB81FC81818FCA
:101D60008091C3078F5F8093C307EB81FC819689C5
:101D70008091BD07891728F4EB81FC8186898093C7
:101D8000BD078B819C81AC014E5F5F4FEB81FC8175
:101D90008689282F3327C901880F991F880F991F1B
:101DA000880F991F820F931F8C53984FBA010E947E
:101DB000771C81E08D830F900FBE02C08FEF8D8363
:101DC0008D818130C1F48F859889009731F0EF853E
:101DD000F8898B819C81918380838091BE078823C1
:101DE00051F0E091B607F091B70796898E85981764
:101DF00010F40E9423238D81992787FD909560968A
:101E00000FB6F894DEBF0FBECDBFDF91CF910F911B
:101E1000FF90EF900895CF93DF93CDB7DEB726976D
:101E20000FB6F894DEBF0FBECDBF9C838B830FB679
:101E3000F8940F922091B6073091B7078B819C815F
:101E40008217930711F41C821B828B819C8100975F
:101E500039F48091B6079091B7079E838D8304C0B3
:101E60008B819C819E838D838D819E819A838983C2
:101E700089819A8102960E94321DE981FA818489C2
:101E80009589009729F089819A810C960E94321DCC
:101E900089819A81029629E138E0BC01C9010E943A
:101EA000771C8091B8078F5F8093B8070F900FBEA3
:101EB0008091BE07882331F08B819C81009711F4BB
:101EC0000E94232326960FB6F894DEBF0FBECDBF27
:101ED000DF91CF910895CF93DF93CDB7DEB72897E9
:101EE0000FB6F894DEBF0FBECDBF9E838D8378877B
:101EF0006F8319820E94AB10ED81FE8120813181B8
:101F00008F819885820F931F9C838B83ED81FE8147
:101F1000208131818091BA079091BB078217930786
:101F2000A8F4ED81FE81208131818B819C81821713
:101F3000930700F52091BA073091BB078B819C81F4
:101F400028173907B8F481E0898314C0ED81FE8138
:101F5000208131818B819C818217930748F02091E9
:101F6000BA073091BB078B819C812817390710F481
:101F700081E08983ED81FE818B819C8191838083C7
:101F80008981882399F18091B6079091B7070296CD
:101F90000E94321DE091B607F091B7078B819C81BA
:101FA000938382832091BA073091BB078B819C81F8
:101FB0008217930770F48091B6079091B707029645
:101FC00020910E0830910F08BC01C9010E94C61C67
:101FD0000DC08091B6079091B707029620910C082A
:101FE00030910D08BC01C9010E94C61C0E94BC10A2
:101FF0008A838A81882311F40E94232328960FB6AE
:10200000F894DEBF0FBECDBFDF91CF910895CF937F
:10201000DF93CDB7DEB725970FB6F894DEBF0FBEBE
:10202000CDBF9D838C8319828C819D81009709F49B
:1020300042C00E94AB102091BA073091BB078C813F
:102040009D81820F931F9B838A838091B607909115
:10205000B70702960E94321DE091B607F091B707CC
:102060008A819B81938382832091BA073091BB0739
:102070008A819B818217930770F48091B6079091B3
:10208000B707029620910E0830910F08BC01C901D4
:102090000E94C61C0DC08091B6079091B7070296AA
:1020A00020910C0830910D08BC01C9010E94C61C8A
:1020B0000E94BC1089838981882311F40E94232304
:1020C00025960FB6F894DEBF0FBECDBFDF91CF913E
:1020D0000895EF92FF920F93CF93DF93CDB7DEB7C2
:1020E00021970FB6F894DEBF0FBECDBF8AEA97E006
:1020F000E7E5F4E1EE24FF2400E020E030E045E5F0
:1021000050E0BC01CF010E942E0E8983898181306D
:1021100051F4F89481E08093BE071092BB071092AF
:10212000BA070E94E62221960FB6F894DEBF0FBED2
:10213000CDBFDF91CF910F91FF90EF900895CF9396
:10214000DF93CDB7DEB7F8941092BE070E941C2330
:10215000DF91CF910895CF93DF93CDB7DEB70FB660
:10216000F8940F928091BF078F5F8093BF070F9005
:102170000FBEDF91CF910895CF93DF93CDB7DEB738
:1021800026970FB6F894DEBF0FBECDBF1A820FB6EA
:10219000F8940F928091BF0781508093BF07809180
:1021A000BF07882309F077C08091B907882309F415
:1021B00072C0198239C08B819C810C960E94321D9D
:1021C0008B819C8102960E94321DEB81FC81968955
:1021D0008091BD07891728F4EB81FC818689809363
:1021E000BD074B815C814E5F5F4FEB81FC8186892F
:1021F000282F3327C901880F991F880F991F880F2F
:10220000991F820F931F8C53984FBA010E94771C1D
:10221000EB81FC819689E091B607F091B70786893A
:10222000981710F081E0898380911008882349F085
:10223000E0911508F0911608868197819E838D8321
:1022400002C01E821D828D819E819C838B83EB81C7
:10225000FC81309709F0AFCF8091C007882371F0DF
:1022600007C00E9497118091C00781508093C007DA
:102270008091C0078823A9F781E089838981813013
:1022800021F08091C107813031F481E08A8310927E
:10229000C1070E9423230F900FBE8A81992787FDD3
:1022A000909526960FB6F894DEBF0FBECDBFDF9196
:1022B000CF910895CF93DF93CDB7DEB722970FB6B6
:1022C000F894DEBF0FBECDBF0FB6F8940F92809189
:1022D000BA079091BB079A8389830F900FBE8981BB
:1022E0009A8122960FB6F894DEBF0FBECDBFDF9164
:1022F000CF910895CF93DF93CDB7DEB721970FB677
:10230000F894DEBF0FBECDBF0FB6F8940F92809148
:10231000B90789830F900FBE8981992721960FB63F
:10232000F894DEBF0FBECDBFDF91CF910895CF935C
:10233000DF93CDB7DEB726970FB6F894DEBF0FBE9A
:10234000CDBF8091BF07882309F088C08091BA076C
:102350009091BB0701969093BB078093BA07809139
:10236000BA079091BB07009709F059C080910C08FB
:1023700090910D089A83898380910E0890910F089F
:1023800090930D0880930C0889819A8190930F088F
:1023900080930E088091C2078F5F8093C2073FC071
:1023A000EB81FC81228133818091BA079091BB0738
:1023B0008217930708F457C08B819C8102960E9474
:1023C000321DEB81FC8184899589009729F08B81EE
:1023D0009C810C960E94321DEB81FC819689809134
:1023E000BD07891728F4EB81FC8186898093BD079E
:1023F0004B815C814E5F5F4FEB81FC818689282F8A
:102400003327C901880F991F880F991F880F991FBB
:10241000820F931F8C53984FBA010E94771CE09152
:102420000C08F0910D088081882361F0E0910C0880
:10243000F0910D080580F681E02D868197819E83BD
:102440008D8302C01E821D828D819E819C838B8321
:10245000EB81FC81309709F0A3CF05C08091C007C4
:102460008F5F8093C00726960FB6F894DEBF0FBE2D
:10247000CDBFDF91CF910895CF93DF93CDB7DEB776
:102480008091BF07882349F081E08093C107A6C0EF
:102490008091BD0781508093BD078091BD07282F93
:1024A0003327C901880F991F880F991F880F991F1B
:1024B000820F931FFC01EC53F84F8081882341F376
:1024C0008091BD07282F3327C901880F991F880FD6
:1024D000991F880F991F820F931FDC01AC53B84FCF
:1024E0008091BD07282F3327C901880F991F880FB6
:1024F000991F880F991F820F931FFC01EC53F84F0F
:102500000180F281E02D82819381FD01928381839C
:102510008091BD07282F3327C901880F991F880F85
:10252000991F880F991F820F931FFC01EC53F84FDE
:10253000418152818091BD07282F3327C901880F1F
:10254000991F880F991F880F991F820F931F8C5313
:10255000984F03964817590741F58091BD07282FDA
:102560003327C901880F991F880F991F880F991F5A
:10257000820F931FDC01AC53B84F8091BD07282F09
:102580003327C901880F991F880F991F880F991F3A
:10259000820F931FFC01EC53F84F0180F281E02D74
:1025A00082819381FD01928381838091BD07282FD1
:1025B0003327C901880F991F880F991F880F991F0A
:1025C000820F931FFC01EC53F84F0180F281E02D44
:1025D000868197819093B7078093B607DF91CF915B
:1025E0000895CF93DF93CDB7DEB726970FB6F89453
:1025F000DEBF0FBECDBF9C838B837E836D838091B6
:10260000B6079091B7070C962B813C81BC01C9019C
:102610000E94C61C8091B6079091B70702960E944F
:10262000321D2091BA073091BB078D819E81820FA8
:10263000931F9A838983E091B607F091B707898148
:102640009A81938382832091BA073091BB07898155
:102650009A818217930770F48091B6079091B7071B
:10266000029620910E0830910F08BC01C9010E940A
:10267000C61C0DC08091B6079091B70702962091B5
:102680000C0830910D08BC01C9010E94C61C269699
:102690000FB6F894DEBF0FBECDBFDF91CF91089586
:1026A000CF93DF93CDB7DEB727970FB6F894DEBF91
:1026B0000FBECDBF9D838C83EC81FD8180818823FB
:1026C00061F08C819D81FC0133960280F381E02DC5
:1026D000868197819F838E8302C01F821E828E8196
:1026E0009F819B838A838A819B810C960E94321DE5
:1026F0008091BF07882351F58A819B8102960E94B1
:10270000321DEA81FB8196898091BD07891728F4E3
:10271000EA81FB8186898093BD078A819B81AC0118
:102720004E5F5F4FEA81FB818689282F3327C901DD
:10273000880F991F880F991F880F991F820F931F69
:102740008C53984FBA010E94771C09C08A819B81E3
:102750000C9620E138E0BC01C9010E94771CEA8197
:10276000FB819689E091B607F091B70786899817A3
:1027700018F081E0898301C019828981992787FD3A
:10278000909527960FB6F894DEBF0FBECDBFDF91B0
:10279000CF910895CF93DF93CDB7DEB722970FB6D1
:1027A000F894DEBF0FBECDBF9A8389838091C207A4
:1027B000E981FA8180838091BA079091BB07E98112
:1027C000FA819283818322960FB6F894DEBF0FBE02
:1027D000CDBFDF91CF910895CF93DF93CDB7DEB713
:1027E00025970FB6F894DEBF0FBECDBF9B838A83BB
:1027F0007D836C83EA81FB8190818091C207981769
:1028000071F0EA81FB81218132818091BA07909138
:10281000BB072817390718F481E0898331C020915C
:10282000BA073091BB07EA81FB8181819281281B25
:10283000390BEC81FD818081918128173907F0F4F3
:10284000EC81FD81408151812091BA073091BB0715
:10285000EA81FB8181819281B901681B790BCB01EF
:102860009A01281B390BC901EC81FD81918380837A
:102870008A819B810E94CA13198202C081E08983E8
:102880008981992787FD909525960FB6F894DEBF2C
:102890000FBECDBFDF91CF910895CF93DF93CDB71A
:1028A000DEB781E08093C107DF91CF910895CF9388
:1028B000DF93CDB7DEB722970FB6F894DEBF0FBE19
:1028C000CDBF9A83898300C00E940B158091C407F5
:1028D0008230D0F30E942323F7CFCF93DF93CDB77D
:1028E000DEB727970FB6F894DEBF0FBECDBF9A8331
:1028F00089837C836B835E834D832F83E981FA8197
:102900008B819C8193A382A32D813E8189819A81B1
:102910004A9648E050E0B9010E947724E981FA81A3
:1029200011A28F81863010F085E08F83E981FA81D2
:102930008F81868B89819A8102960E945E1C898193
:102940009A810C960E945E1CE981FA8189819A81A4
:10295000918780878F81282F332786E090E0821B24
:10296000930BE981FA8195878487E981FA818981CE
:102970009A81938B828B27960FB6F894DEBF0FBE99
:10298000CDBFDF91CF910895CF93DF93CDB7DEB761
:1029900021970FB6F894DEBF0FBECDBF198213C0CA
:1029A0008981282F3327C901880F991F880F991F04
:1029B000880F991F820F931F8C53984F0E942B1CD6
:1029C00089818F5F89838981863050F38AEF97E010
:1029D0000E942B1C83E098E00E942B1C80E198E071
:1029E0000E942B1C89E198E00E942B1C8AEF97E043
:1029F00090930D0880930C0883E098E090930F0863
:102A000080930E0821960FB6F894DEBF0FBECDBF9F
:102A1000DF91CF910895CF93DF93CDB7DEB72597A0
:102A20000FB6F894DEBF0FBECDBF8091B8078823E4
:102A300009F43DC00E94AB10809119081B828823C5
:102A400011F481E08B830E94BC108B81882379F57F
:102A50000FB6F8940F92E9E1F8E08081882361F0E5
:102A600089E198E0FC0133960280F381E02D8681B4
:102A700097819D838C8302C01D821C828C819D81E5
:102A80009A83898389819A8102960E94321D80915E
:102A9000B90781508093B9078091B807815080931E
:102AA000B8070F900FBE89819A810E94A2152596C2
:102AB0000FB6F894DEBF0FBECDBFDF91CF91089562
:102AC000CF93DF93CDB7DEB724970FB6F894DEBF70
:102AD0000FBECDBF9C838B8384E290E00E94E820F0
:102AE0009A83898389819A81009709F18B819C81DE
:102AF0000E94E820E981FA81908F878BE981FA8131
:102B00008789908D009739F489819A810E943421B8
:102B10001A8219820CC0E981FA812789308D8B8154
:102B20009C81AC0165EA70E0C9010E947024898132
:102B30009A8124960FB6F894DEBF0FBECDBFDF9109
:102B4000CF910895CF93DF93CDB7DEB722970FB61D
:102B5000F894DEBF0FBECDBF9A838983E981FA81E5
:102B60008789908D0E94342189819A810E94342125
:102B700022960FB6F894DEBF0FBECDBFDF91CF9186
:102B80000895CF93DF93CDB7DEB728970FB6F894AB
:102B9000DEBF0FBECDBF8D836E838D81882309F488
:102BA00088C08FE190E00E94E8209C838B838B811A
:102BB0009C81009709F47DC08D81282F33278E8159
:102BC0009927AC01249FC001259F900D349F900D43
:102BD000112401969A83898389819A810E94E82031
:102BE000EB81FC8191838083EB81FC8180819181E9
:102BF000009709F45AC0EB81FC81408151818D819D
:102C0000282F33278E819927BC01269FC001279F3B
:102C1000900D369F900D1124840F951FEB81FC8140
:102C200093838283EB81FC81128EEB81FC81808116
:102C30009181EB81FC8195838483EB81FC814081D0
:102C400051818D8199279C01215030408E81992797
:102C5000BC01269FC001279F900D369F900D112427
:102C6000840F951FEB81FC8197838683EB81FC8128
:102C70008D81838FEB81FC818E81848FEB81FC8140
:102C80008FEF858FEB81FC818FEF868F8B819C810D
:102C900008960E942B1C8B819C8141960E942B1CC4
:102CA0008B819C8198878F8306C08B819C810E9439
:102CB000342118861F828F81988528960FB6F89444
:102CC000DEBF0FBECDBFDF91CF910895CF93DF93CD
:102CD000CDB7DEB72A970FB6F894DEBF0FBECDBFD3
:102CE0009E838D8378876F835A8749870E94AB10B4
:102CF000CE0102960E94CA130FB6F8940F92ED818E
:102D0000FE81858D8F5FED81FE81858FED81FE8156
:102D1000868D8F5FED81FE81868F0F900FBE8D8136
:102D20009E810E94E619882381F189859A85009702
:102D300061F129853A858D819E810896B9010E94AD
:102D4000F1120FB6F8940F928D819E810E94631943
:102D50000E94BC10882311F40E9423230E94AB1010
:102D60000FB6F8940F92ED81FE81858D8F5FED8116
:102D7000FE81858FED81FE81868D8F5FED81FE81E5
:102D8000868F0F900FBE0F900FBE0FB6F8940F9264
:102D9000ED81FE81928DED81FE81838D981708F083
:102DA00044C0ED81FE81848D482F5527ED81FE8141
:102DB000848195812F813885FC01CA01AC01B9015C
:102DC000CF010E946724ED81FE81828D8F5FED81AE
:102DD000FE81828FED81FE8124813581ED81FE812E
:102DE000848D9927820F931FED81FE8195838483C3
:102DF000ED81FE8124813581ED81FE818281938187
:102E00002817390740F0ED81FE8180819181ED81A5
:102E1000FE819583848381E08983ED81FE81868DA7
:102E20008F5FED81FE81868F01C019820F900FBEEA
:102E30008981882389F489859A85009769F0CE0174
:102E400009969E012E5F3F4FBC01C9010E94EC1301
:102E5000882311F48FEF898389818F3F09F45FCF35
:102E60008D819E810E9463190E94BC1089819927DF
:102E700087FD90952A960FB6F894DEBF0FBECDBFA2
:102E8000DF91CF910895CF93DF93CDB7DEB727972A
:102E90000FB6F894DEBF0FBECDBF9A8389837C83C3
:102EA0006B834D83E981FA81928DE981FA81838D6B
:102EB000981708F05AC0E981FA81848D482F552768
:102EC000E981FA81848195812B813C81FC01CA01D1
:102ED000AC01B901CF010E946724E981FA81828D9A
:102EE0008F5FE981FA81828FE981FA8124813581BE
:102EF000E981FA81848D9927820F931FE981FA81F4
:102F000095838483E981FA8124813581E981FA817D
:102F1000828193812817390740F0E981FA81808105
:102F20009181E981FA8195838483E981FA81868D93
:102F30008F3FA1F48D818823C1F4E981FA818189D1
:102F4000882399F089819A8141960E9450138823A1
:102F500061F021E030E03F832E830EC0E981FA81E9
:102F6000868D8F5FE981FA81868F8D81282F3327A7
:102F700027FD30953F832E838E819F8127960FB644
:102F8000F894DEBF0FBECDBFDF91CF910895CF93F0
:102F9000DF93CDB7DEB72A970FB6F894DEBF0FBE2A
:102FA000CDBF9E838D8378876F835A8749870E9420
:102FB000AB10CE0102960E94CA130FB6F8940F927E
:102FC000ED81FE81858D8F5FED81FE81858FED81A5
:102FD000FE81868D8F5FED81FE81868F0F900FBE03
:102FE0008D819E810E94C019882381F189859A85EF
:102FF000009761F129853A858D819E814196B901BD
:103000000E94F1120FB6F8940F928D819E810E945A
:1030100063190E94BC10882311F40E9423230E948C
:10302000AB100FB6F8940F92ED81FE81858D8F5F06
:10303000ED81FE81858FED81FE81868D8F5FED8133
:10304000FE81868F0F900FBE0F900FBE0FB6F894C3
:103050000F92ED81FE81828D882309F444C0ED81B9
:10306000FE8126813781ED81FE81848D9927820F33
:10307000931FED81FE8197838683ED81FE812681FA
:103080003781ED81FE81828193812817390740F0D5
:10309000ED81FE8180819181ED81FE819783868320
:1030A000ED81FE81828D8150ED81FE81828FED81E7
:1030B000FE81848D482F5527ED81FE812681378141
:1030C0008F819885FC01CA01AC01B901CF010E9432
:1030D0006724ED81FE81858D8F5FED81FE81858F77
:1030E00081E0898301C019820F900FBE89818823F6
:1030F00089F489859A85009769F0CE0109969E0129
:103100002E5F3F4FBC01C9010E94EC13882311F4CC
:103110008FEF898389818F3F09F462CF8D819E81F2
:103120000E9463190E94BC108981992787FD9095A0
:103130002A960FB6F894DEBF0FBECDBFDF91CF91B8
:103140000895CF93DF93CDB7DEB727970FB6F894E6
:10315000DEBF0FBECDBF9B838A837D836C835F837D
:103160004E83EA81FB81828D882309F45FC0EA8166
:10317000FB8126813781EA81FB81848D9927820F2B
:10318000931FEA81FB8197838683EA81FB812681F5
:103190003781EA81FB81828193812817390740F0CA
:1031A000EA81FB8180819181EA81FB81978386831B
:1031B000EA81FB81828D8150EA81FB81828FEA81E5
:1031C000FB81848D482F5527EA81FB812681378139
:1031D0008C819D81FC01CA01AC01B901CF010E9423
:1031E0006724EA81FB81858D8F3FB1F4EE81FF81F9
:1031F00080818823C1F4EA81FB818085882399F04E
:103200008A819B8108960E945013882361F0EE8189
:10321000FF8181E0808307C0EA81FB81858D8F5F1C
:10322000EA81FB81858F81E0898301C019828981D0
:10323000992787FD909527960FB6F894DEBF0FBEAD
:10324000CDBFDF91CF910895CF93DF93CDB7DEB798
:1032500023970FB6F894DEBF0FBECDBF9B838A8342
:103260000FB6F8940F92EA81FB81828D89830F90CB
:103270000FBE8981992723960FB6F894DEBF0FBE43
:10328000CDBFDF91CF910895CF93DF93CDB7DEB758
:1032900022970FB6F894DEBF0FBECDBF9A83898305
:1032A000E981FA81808191810E94342189819A810A
:1032B0000E94342122960FB6F894DEBF0FBECDBF18
:1032C000DF91CF910895CF93DF93CDB7DEB72297EB
:1032D0000FB6F894DEBF0FBECDBF9A8389830FB6B9
:1032E000F8940F92E981FA81868D8150E981FA8103
:1032F000868FE981FA81868D8F3F99F094F0E9817C
:10330000FA818FEF868FE981FA818189882349F0DC
:1033100089819A8141960E945013882311F00E945E
:103320004D140F900FBE0FB6F8940F92E981FA81F9
:10333000858D8150E981FA81858FE981FA81858DBA
:103340008F3F99F094F0E981FA818FEF858FE981C1
:10335000FA818085882349F089819A8108960E94A4
:103360005013882311F00E944D140F900FBE229627
:103370000FB6F894DEBF0FBECDBFDF91CF91089599
:10338000CF93DF93CDB7DEB723970FB6F894DEBFA8
:103390000FBECDBF9B838A830FB6F8940F92EA814C
:1033A000FB81828D1982882311F481E089830F903B
:1033B0000FBE8981992787FD909523960FB6F894C3
:1033C000DEBF0FBECDBFDF91CF910895CF93DF93C6
:1033D000CDB7DEB723970FB6F894DEBF0FBECDBFD3
:1033E0009B838A830FB6F8940F92EA81FB81928DBA
:1033F000EA81FB81838D1982981711F481E089831A
:103400000F900FBE8981992787FD909523960FB65F
:10341000F894DEBF0FBECDBFDF91CF910895CF935B
:10342000DF93CDB7DEB729970FB6F894DEBF0FBE96
:10343000CDBF9B838A837D836C835F834E83F894A7
:103440008A819B810E94E6198823B9F08E819F8131
:10345000009779F08A819B8108962E813F81BC017B
:10346000C9010E94141E78942CEF3FEF39872887FA
:1034700064C078941986188660C078940000F89427
:10348000EA81FB81928DEA81FB81838D981708F098
:103490004BC0EA81FB81848D482F5527EA81FB814F
:1034A000848195812C813D81FC01CA01AC01B90167
:1034B000CF010E946724EA81FB81828D8F5FEA81C0
:1034C000FB81828FEA81FB8124813581EA81FB8146
:1034D000848D9927820F931FEA81FB8195838483D2
:1034E000EA81FB8124813581EA81FB81828193819C
:1034F0002817390740F0EA81FB8180819181EA81B8
:10350000FB819583848381E08983EA81FB818189C2
:10351000882359F08A819B8141960E949C208823B0
:1035200021F08BEF898301C0198278948981282F3B
:10353000332727FD309539872887888599852996EF
:103540000FB6F894DEBF0FBECDBFDF91CF910895C7
:10355000CF93DF93CDB7DEB729970FB6F894DEBFD0
:103560000FBECDBF9B838A837D836C835F834E8335
:10357000F894EA81FB81828D8823B9F48E819F8142
:10358000009779F08A819B8141962E813F81BC0111
:10359000C9010E94141E78942CEF3FEF39872887C9
:1035A00061C07894198618865DC078940000F894FC
:1035B000EA81FB81828D882309F44BC0EA81FB817B
:1035C00026813781EA81FB81848D9927820F931FA1
:1035D000EA81FB8197838683EA81FB81268137819B
:1035E000EA81FB81828193812817390740F0EA81C3
:1035F000FB8180819181EA81FB8197838683EA81C7
:10360000FB81828D8150EA81FB81828FEA81FB817F
:10361000848D482F5527EA81FB81268137818C8153
:103620009D81FC01CA01AC01B901CF010E94672450
:1036300081E08983EA81FB818085882359F08A8132
:103640009B8108960E949C20882321F08BEF898320
:1036500001C0198278948981282F332727FD30955E
:10366000398728878885998529960FB6F894DEBF13
:103670000FBECDBFDF91CF910895CF93DF93CDB72C
:10368000DEB727970FB6F894DEBF0FBECDBF9A8383
:1036900089837C836B834D83E981FA81928DE981F3
:1036A000FA81838D981708F04EC0E981FA81848DE4
:1036B000482F5527E981FA81848195812B813C81AE
:1036C000FC01CA01AC01B901CF010E946724E98164
:1036D000FA81828D8F5FE981FA81828FE981FA8197
:1036E00024813581E981FA81848D9927820F931F86
:1036F000E981FA8195838483E981FA812481358186
:10370000E981FA81828193812817390740F0E981A4
:10371000FA8180819181E981FA81958384838D8109
:10372000882389F4E981FA818189882361F089817C
:103730009A8141960E949C20882329F021E030E064
:103740003F832E8307C08D81282F332727FD309597
:103750003F832E838E819F8127960FB6F894DEBF1C
:103760000FBECDBFDF91CF910895CF93DF93CDB73B
:10377000DEB727970FB6F894DEBF0FBECDBF9B8391
:103780008A837D836C835F834E83EA81FB81828D94
:10379000882309F452C0EA81FB8126813781EA81BE
:1037A000FB81848D9927820F931FEA81FB81978388
:1037B0008683EA81FB8126813781EA81FB818281D0
:1037C00093812817390740F0EA81FB81808191813C
:1037D000EA81FB8197838683EA81FB81828D815018
:1037E000EA81FB81828FEA81FB81848D482F5527F6
:1037F000EA81FB81268137818C819D81FC01CA0190
:10380000AC01B901CF010E946724EE81FF81808164
:10381000882381F4EA81FB818085882359F08A819D
:103820009B8108960E949C20882321F0EE81FF81D5
:1038300081E0808381E0898301C019828981992791
:1038400087FD909527960FB6F894DEBF0FBECDBFCB
:10385000DF91CF910895CF93DF93CDB7DEB7229755
:103860000FB6F894DEBF0FBECDBF9A8389838981DE
:103870009A810396E981FA8192838183E981FA81B1
:103880008FEF9FEF9483838389819A810396E981E7
:10389000FA819683858389819A810396E981FA81E9
:1038A00090878783E981FA81108222960FB6F89477
:1038B000DEBF0FBECDBFDF91CF910895CF93DF93D1
:1038C000CDB7DEB722970FB6F894DEBF0FBECDBFDF
:1038D0009A838983E981FA811186108622960FB630
:1038E000F894DEBF0FBECDBFDF91CF910895CF9387
:1038F000DF93CDB7DEB726970FB6F894DEBF0FBEC5
:10390000CDBF9C838B837E836D83EB81FC81818122
:1039100092819A838983E981FA8182819381ED8101
:10392000FE8193838283EB81FC8181819281ED8191
:10393000FE8195838483E981FA810280F381E02D01
:103940008D819E81958384838D819E81E981FA8119
:10395000938382838D819E81EB81FC81928381831D
:10396000ED81FE818B819C8191878087EB81FC8139
:1039700080818F5FEB81FC81808326960FB6F8945F
:10398000DEBF0FBECDBFDF91CF910895CF93DF9300
:10399000CDB7DEB728970FB6F894DEBF0FBECDBF08
:1039A0009E838D8378876F83EF81F88580819181F5
:1039B0009A83898389819A812FEF8F3F920739F407
:1039C000ED81FE81878190859C838B8318C08D81DA
:1039D0009E8103969C838B8306C0EB81FC81828150
:1039E00093819C838B83EB81FC810280F381E02DAA
:1039F0002081318189819A818217930770F7EB8149
:103A0000FC8182819381EF81F88593838283EF81AA
:103A1000F8850280F381E02D8F81988595838483DA
:103A2000EF81F8858B819C81958384838F81988534
:103A3000EB81FC8193838283EF81F8858D819E8168
:103A400091878087ED81FE8180818F5FED81FE818E
:103A5000808328960FB6F894DEBF0FBECDBFDF91EE
:103A6000CF910895CF93DF93CDB7DEB724970FB6EC
:103A7000F894DEBF0FBECDBF9C838B83EB81FC81AE
:103A8000A281B381EB81FC8184819581FD019583C5
:103A90008483EB81FC81A481B581EB81FC818281EF
:103AA0009381FD0193838283EB81FC8180859185E5
:103AB0009A838983E981FA81218132818B819C817A
:103AC0002817390741F4EB81FC8184819581E981D4
:103AD000FA8192838183EB81FC8111861086E981D2
:103AE000FA8180818150E981FA81808324960FB622
:103AF000F894DEBF0FBECDBFDF91CF910895CF9375
:103B0000DF93CDB7DEB727970FB6F894DEBF0FBEB1
:103B1000CDBF9D838C836E834F838AE190E00E94AA
:103B2000E8209A83898389819A81009709F46DC07E
:103B30008091220890912308009741F489819A810D
:103B400090932308809322080E9459208E8182300E
:103B500010F081E08E83E981FA81118E108EE98167
:103B6000FA818E81868BE981FA818F81878BE98149
:103B7000FA818C819D819183808389819A810296CB
:103B80000E945E1C89819A810C960E945E1CE981CC
:103B9000FA8189819A8191878087E981FA81898177
:103BA0009A81938B828B8E81282F332786E090E039
:103BB000821B930BE981FA8195878487E981FA81D9
:103BC000968980912408891728F4E981FA818689E9
:103BD0008093240889819A81AC014E5F5F4FE9810F
:103BE000FA818689282F3327C901880F991F880FEA
:103BF000991F880F991F820F931F855D974FBA01F8
:103C00000E94771C81E08B8302C08FEF8B838B81B6
:103C1000992787FD909527960FB6F894DEBF0FBEC3
:103C2000CDBFDF91CF910895CF93DF93CDB7DEB7AE
:103C300026970FB6F894DEBF0FBECDBF9C838B8353
:103C40007E836D8320912508309126088B819C818D
:103C5000820F931F9A838983809122089091230871
:103C600002960E94321DE0912208F091230889817A
:103C70009A81938382832091250830912608898137
:103C80009A818217930770F48091220890912308FB
:103C900002962091510830915208BC01C9010E943E
:103CA000C61C0DC080912208909123080296209195
:103CB0004F0830915008BC01C9010E94C61C8D817B
:103CC0009E81009759F080912208909123080C96CC
:103CD0002D813E81BC01C9010E94C61C26960FB6EB
:103CE000F894DEBF0FBECDBFDF91CF910895CF9383
:103CF000DF93CDB7DEB70E94401F0E949C1F0AC011
:103D000080912408882309F4B8C080912408815048
:103D10008093240880912408282F3327C901880F15
:103D2000991F880F991F880F991F820F931FFC01FD
:103D3000E55DF74F8081882319F380912408282FAF
:103D40003327C901880F991F880F991F880F991F62
:103D5000820F931FDC01A55DB74F80912408282FA7
:103D60003327C901880F991F880F991F880F991F42
:103D7000820F931FFC01E55DF74F0180F281E02D7A
:103D800082819381FD019283818380912408282F71
:103D90003327C901880F991F880F991F880F991F12
:103DA000820F931FFC01E55DF74F418152818091A5
:103DB0002408282F3327C901880F991F880F991FBE
:103DC000880F991F820F931F855D974F03964817A1
:103DD000590741F580912408282F3327C901880FFE
:103DE000991F880F991F880F991F820F931FDC015D
:103DF000A55DB74F80912408282F3327C901880F6C
:103E0000991F880F991F880F991F820F931FFC011C
:103E1000E55DF74F0180F281E02D82819381FD0104
:103E20009283818380912408282F3327C901880F2A
:103E3000991F880F991F880F991F820F931FFC01EC
:103E4000E55DF74F0180F281E02D868197819093A7
:103E5000230880932208E0912208F09123084081F2
:103E60005181E0912208F09123082789809122084E
:103E700090912308622FFA011995DF91CF9108954F
:103E8000CF93DF93CDB7DEB724970FB6F894DEBF9C
:103E90000FBECDBF43C0F89480915308882349F0EA
:103EA000E0915808F0915908868197819C838B8313
:103EB00002C01C821B828B819C819A8389838981A9
:103EC0009A810C960E94321D789489819A8102967B
:103ED0000E94321DE981FA81968980912408891710
:103EE00028F4E981FA8186898093240889819A815E
:103EF000AC014E5F5F4FE981FA818689282F332715
:103F0000C901880F991F880F991F880F991F820F69
:103F1000931F855D974FBA010E94771C80915308CB
:103F2000882309F0B8CF24960FB6F894DEBF0FBEF1
:103F3000CDBFDF91CF910895CF93DF93CDB7DEB79B
:103F400026970FB6F894DEBF0FBECDBF0E945A1160
:103F50002091290830912A08821B930B90932808FE
:103F6000809327088EC0809125089091260801969D
:103F7000909326088093250880912708909128081F
:103F800001979093280880932708809125089091A5
:103F90002608009709F057C080914F08909150086B
:103FA0009A83898380915108909152089093500888
:103FB00080934F0889819A81909352088093510889
:103FC00042C0EB81FC812281338180912508909150
:103FD00026088217930708F454C0F8948B819C81BB
:103FE00002960E94321DEB81FC818489958900979D
:103FF00029F08B819C810C960E94321D7894EB8174
:10400000FC81968980912408891728F4EB81FC8132
:104010008689809324088B819C81AC014E5F5F4F21
:10402000EB81FC818689282F3327C901880F991FCE
:10403000880F991F880F991F820F931F855D974FD7
:10404000BA010E94771CE0914F08F09150088081DE
:10405000882361F0E0914F08F09150080580F681C7
:10406000E02D868197819E838D8302C01E821D82F2
:104070008D819E819C838B838B819C81009709F02D
:10408000A0CF8091270890912808009709F06BCF66
:10409000809125089091260890932A0880932908FA
:1040A00026960FB6F894DEBF0FBECDBFDF91CF913D
:1040B0000895CF93DF93CDB7DEB721970FB6F8946D
:1040C000DEBF0FBECDBF198213C08981282F3327D1
:1040D000C901880F991F880F991F880F991F820F98
:1040E000931F855D974F0E942B1C89818F5F898369
:1040F0008981823050F38DE398E00E942B1C86E486
:1041000098E00E942B1C83E598E00E942B1C8DE315
:1041100098E09093500880934F0886E498E090933D
:1041200052088093510821960FB6F894DEBF0FBE57
:10413000CDBFDF91CF910895CF93DF93CDB7DEB799
:1041400027970FB6F894DEBF0FBECDBF9D838C833B
:10415000EC81FD818081882361F08C819D81FC014F
:1041600033960280F381E02D868197819F838E8331
:1041700002C01F821E828E819F819B838A838A81D7
:104180009B810C960E94321D8A819B810C9623E5AF
:1041900038E0BC01C9010E94771CEA81FB81968945
:1041A000E0912208F09123088689981718F081E0A1
:1041B000898301C019828981992787FD9095279667
:1041C0000FB6F894DEBF0FBECDBFDF91CF9108953B
:1041D000CF93DF93CDB7DEB724970FB6F894DEBF49
:1041E0000FBECDBF9C838B831A8219820E94AB10B5
:1041F00080915C0890915D082B813C81820F931F18
:1042000029E0843C920718F520915C0830915D0804
:104210008B819C81280F391F80915C0890915D08EB
:1042200082179307A0F480915C0890915D088E59E5
:10423000974F9A83898320915C0830915D088B8128
:104240009C81820F931F90935D0880935C080E946D
:10425000BC1089819A8124960FB6F894DEBF0FBEF8
:10426000CDBFDF91CF910895CF93DF93CDB7DEB768
:1042700022970FB6F894DEBF0FBECDBF9A83898315
:1042800022960FB6F894DEBF0FBECDBFDF91CF915F
:104290000895CF93DF93CDB7DEB710925D081092EB
:1042A0005C08DF91CF910895CF93DF93CDB7DEB750
:1042B00028970FB6F894DEBF0FBECDBF9C838B83CB
:1042C0007E836D8358874F83EB81FC8181E18083FE
:1042D0008B819C8101979C838B83EB81FC8182E2A3
:1042E00080838B819C8101979C838B83EB81FC81F4
:1042F00083E380838B819C8101979C838B838D8159
:104300009E819A8389838981EB81FC8180838B8163
:104310009C8101979C838B8389819A81892F99271E
:104320009A8389838981EB81FC8180838B819C8145
:1043300001979C838B8389819A81892F99279A83FE
:1043400089838981EB81FC8180838B819C810197AA
:104350009C838B83EB81FC8110828B819C810197F4
:104360009C838B83EB81FC8180E880838B819C81A3
:1043700001979C838B83EB81FC8110828B819C81D4
:1043800001979C838B83EB81FC8182E080838B810E
:104390009C8101979C838B83EB81FC8183E08083EC
:1043A0008B819C8101979C838B83EB81FC8184E0D2
:1043B00080838B819C8101979C838B83EB81FC8123
:1043C00085E080838B819C8101979C838B83EB812B
:1043D000FC8186E080838B819C8101979C838B8309
:1043E000EB81FC8187E080838B819C8101979C839A
:1043F0008B83EB81FC8188E080838B819C8101979A
:104400009C838B83EB81FC8189E080838B819C8101
:1044100001979C838B83EB81FC8180E180838B817E
:104420009C8101979C838B83EB81FC8181E180835C
:104430008B819C8101979C838B83EB81FC8182E142
:1044400080838B819C8101979C838B83EB81FC8192
:1044500083E180838B819C8101979C838B83EB819B
:10446000FC8184E180838B819C8101979C838B8379
:10447000EB81FC8185E180838B819C8101979C830A
:104480008B83EB81FC8186E180838B819C8101970A
:104490009C838B83EB81FC8187E180838B819C8172
:1044A00001979C838B83EB81FC8188E180838B81E6
:1044B0009C8101979C838B83EB81FC8189E18083C4
:1044C0008B819C8101979C838B83EB81FC8180E2B3
:1044D00080838B819C8101979C838B83EB81FC8102
:1044E00081E280838B819C8101979C838B83EB810C
:1044F000FC8182E280838B819C8101979C838B83EA
:10450000EB81FC8183E280838B819C8101979C837A
:104510008B838F8198859A8389838981EB81FC8144
:1045200080838B819C8101979C838B8389819A8175
:10453000892F99279A8389838981EB81FC818083E4
:104540008B819C8101979C838B83EB81FC8186E22C
:1045500080838B819C8101979C838B83EB81FC8181
:1045600087E280838B819C8101979C838B83EB8185
:10457000FC8188E280838B819C8101979C838B8363
:10458000EB81FC8189E280838B819C8101979C83F4
:104590008B83EB81FC8180E380838B819C810197FD
:1045A0009C838B83EB81FC8181E380838B819C8165
:1045B00001979C838B838B819C8128960FB6F894FE
:1045C000DEBF0FBECDBFDF91CF910895CF93DF93B4
:1045D000CDB7DEB70E94D723A091B607B091B70739
:1045E000CD91CDBFDD91DEBFFF91EF91DF91CF91F6
:1045F000BF91AF919F918F917F916F915F914F91FB
:104600003F912F911F910F91FF90EF90DF90CF90EE
:10461000BF90AF909F908F907F906F905F904F90E2
:104620003F902F901F900F900FBE0F90089581E044
:1046300090E0DF91CF910895CF93DF93CDB7DEB7B0
:10464000DF91CF9108950F920FB6F8940F921F92B9
:1046500011242F923F924F925F926F927F928F928E
:104660009F92AF92BF92CF92DF92EF92FF920F9301
:104670001F932F933F934F935F936F937F938F93EA
:104680009F93AF93BF93CF93DF93EF93FF93A0914B
:10469000B607B091B7070DB60D920EB60D920E94F7
:1046A0003C12A091B607B091B707CD91CDBFDD9177
:1046B000DEBFFF91EF91DF91CF91BF91AF919F91BD
:1046C0008F917F916F915F914F913F912F911F91AA
:1046D0000F91FF90EF90DF90CF90BF90AF909F90A1
:1046E0008F907F906F905F904F903F902F901F9092
:1046F0000F900FBE0F9008950F920FB6F8940F927F
:104700001F9211242F923F924F925F926F927F924D
:104710008F929F92AF92BF92CF92DF92EF92FF92D1
:104720000F931F932F933F934F935F936F937F93B9
:104730008F939F93AF93BF93CF93DF93EF93FF93A9
:10474000A091B607B091B7070DB60D920EB60D92B7
:104750000E9497110E943C12A091B607B091B70732
:10476000CD91CDBFDD91DEBFFF91EF91DF91CF9174
:10477000BF91AF919F918F917F916F915F914F9179
:104780003F912F911F910F91FF90EF90DF90CF906D
:10479000BF90AF909F908F907F906F905F904F9061
:1047A0003F902F901F900F900FBE0F900895CF93C2
:1047B000DF93CDB7DEB726970FB6F894DEBF0FBEF6
:1047C000CDBF80E89EE3A0E0B0E08B839C83AD8307
:1047D000BE838B819C81AD81BE81689415F8B695AE
:1047E000A795979587951694D1F78B839C83AD8376
:1047F000BE838B819C81AD81BE810197A109B109E6
:104800008B839C83AD83BE838B8189838B819C81C9
:10481000AD81BE81892F9A2FAB2FBB278B839C83C1
:10482000AD83BE838B818A83E9E8F0E08A8180834F
:10483000E8E8F0E089818083A0E8B0E0E0E8F0E01B
:1048400080818C728C93E1E8F0E08BE08083AFE6AE
:10485000B0E0EFE6F0E0808182608C9326960FB6A0
:10486000F894DEBF0FBECDBFDF91CF9108950E94B7
:104870007C231895FC0188279927E894219122230D
:10488000F1F02032D9F32930C9F32A30B9F32C30B2
:10489000A9F32D3099F3263789F32B3219F02D32F5
:1048A00021F468942191222351F0203344F02A33DB
:1048B00034F420530E94A724820F911DF3CF811559
:1048C000910521F01EF48095909501960895FB01C5
:1048D000DC0102C001900D9241505040D8F708957C
:1048E000DC0101C06D9341505040E0F70895FB0199
:1048F000DC014150504048F001900D920020C9F772
:1049000001C01D9241505040E0F70895FB019F0106
:10491000E8944230C4F04532B4F44A3029F497FBAD
:104920001EF4909581959F4F642F77270E94B325A1
:10493000805D8A330CF0895D8193CB010097A1F7EC
:1049400016F45DE251931082C9010C94AF247AE011
:10495000979F902D879F802D910D11240895DC0144
:10496000FC0101900020E9F73297AE17BF0730F441
:104970007C916081708331976D93F7CF0895505883
:10498000192EC1D001D0A4C0BA17620773078407DB
:104990009507B1F188F40EF410940B2EBA2FA02DC8
:1049A000062E622F202D072E732F302D082E842FD8
:1049B000402D092E952F502DFF275523B9F0591B57
:1049C00049F0573E98F0469537952795A795F040C2
:1049D0005395C9F776F0BA0F621F731F841F30F426
:1049E000879577956795B795F040939517FA0F2EB1
:1049F0000895BF1BBB27BA0B620B730B840BF6CF5A
:104A0000DEF6AFC080D001D063C0552359F09923A2
:104A100069F09F575F57951B33F442F4903811F4B7
:104A2000915805C06DC091589F3F09F49AC0BB27AB
:104A3000112462177307840730F4660F771F881FED
:104A4000BB1F915098F311D00F920FD00F920DD041
:104A5000A0E82617370748071B0609F0A048BA2F19
:104A6000602D7F918F9100240895A0E800246217A3
:104A700073078407B10528F0621B730B840BB1091F
:104A80000A2A660F771F881FBB1FA69581F7089516
:104A900097FB45D09F3738F0FEE9F91B982F872FF9
:104AA000762F6B2F05C05AC0969587957795679599
:104AB000F150D0F73EF490958095709561957F4FB9
:104AC0008F4F9F4F08959A95BB0F661F771F881FC2
:104AD00011249923A1F08823B2F79F3F59F0BB0F0F
:104AE00048F421F4002011F460FF04C06F5F7F4F91
:104AF0008F4F9F4F881F9795879597F908952EC0E0
:104B00009FEF80EC0895052E092607FA440F551FE4
:104B10005F3F79F0AA27A51708F051E04795880F65
:104B2000991F9F3F31F0BB27B91708F091E0879597
:104B300008959F919F919F911124E2CF97FB880F39
:104B4000991F9F3F31F0BB27B91708F091E0879577
:104B500008959F919F919F911124D2CF6627772727
:104B6000882799270895AA1BBB1B51E107C0AA1FDC
:104B7000BB1FA617B70710F0A61BB70B881F991FFE
:0E4B80005A95A9F780959095BC01CD01089536
:104B8E009001FF01010100466C6173684F4B004DAF
:104B9E00656E7500576174636854656D70000D0A1B
:104BAE005741524E494E473A20554E495420544F84
:104BBE004F20484F542E0D0A5374616E6462792053
:104BCE00666F7220636F6F6C20646F776E2C207728
:104BDE00696C6C20726573756D65206175746F6D8F
:104BEE0061746963616C6C79207768656E2073619E
:104BFE0066652E2E2E0000526573756D696E672EDA
:104C0E000D0A000D0A0D0A0D0A0D0A0D0A0D0A0DE8
:104C1E000A0D0A0D0A0D0A0D0A0D0A004D756C7467
:104C2E0069737065637472616C20496C6C756D6923
:104C3E006E61746F720D0A4669726D7761726520CE
:104C4E0056657273696F6E20312E300D0A00004F5B
:104C5E004B00004572726F723A204D696E696D7528
:104C6E006D2074696D65206265747765656E20735D
:104C7E00686F747320697320356D732E0000457252
:104C8E00726F723A204D6178696D756D2073686F21
:104C9E0074732070657220636F6C6F72206973205D
:104CAE003235352E00004572726F723A204D696EA4
:104CBE00696D756D206E756D626572206F662073FD
:104CCE00686F74732070657220636F6C6F722069E9
:104CDE007320312E00004572726F723A2043686164
:104CEE006E6E656C206E756D626572206D75737477
:104CFE00206265206265747765656E203120616E75
:104D0E0064203920696E636C75736976652E0000B8
:104D1E004572726F723A2053657175656E636520C8
:104D2E006D75737420657865637574652061742084
:104D3E006C65617374206F6E63652E000009437598
:104D4E007272656E7420486F7420506C61746520A9
:104D5E0054656D70657261747572653A200000431A
:104D6E000D0A00000943757272656E74205043423D
:104D7E00204578746572696F722054656D70657226
:104D8E0061747572653A2000004572726F723A2036
:104D9E00556E6B6E6F776E20436F6D6D616E642E08
:104DAE00205072657373203F20666F722068656CA9
:104DBE00702E00000D0A436F6D6D616E64204865A4
:104DCE006C703A0D0A00002D2D2D2D2D2D2D2D2D13
:104DDE002D2D2D2D0D0A00003F0953686F7720747D
:104DEE006869732068656C70206D656E750D0A00BC
:104DFE000070095072696E7420636F6E6669677514
:104E0E00726174696F6E0D0A0000670953686F6FE7
:104E1E00742073657175656E6365206F66207069A9
:104E2E0063747572657320617320636F6E66696754
:104E3E00757265640D0A00006D6E094D6972726FB0
:104E4E0072206C6F636B75702064656C6179202DB8
:104E5E002035306D532C206F72203020746F2064FB
:104E6E00697361626C6520286E2075732064656CB1
:104E7E00617920696E206D7329205B305D0D0A000B
:104E8E0000776E0953657420776169742074696DBB
:104E9E006520666F7220656163682063616D65725F
:104EAE0061206669726520286E2069732074696DB1
:104EBE006520696E206D7329205B3430305D0D0ADC
:104ECE000000236E094E756D626572206F66206359
:104EDE00616D6572612073686F74732070657220E6
:104EEE00636F6C6F7220286E206973206E756D6211
:104EFE006572206F662073686F747329205B315D55
:104F0E000D0A0000456E09456E61626C6520636F87
:104F1E006C6F72206E20666F722073657175656E90
:104F2E0063650D0A0000446E0944697361626C6525
:104F3E0020636F6C6F72206E20666F7220736571C6
:104F4E0075656E63650D0A0000726E0952657065B7
:104F5E006174207468652073657175656E63652074
:104F6E006E2074696D65730D0A00007409446973CF
:104F7E00706C61792054656D7065726174757265BF
:104F8E00730D0A00000D0A43757272656E7420432C
:104F9E006F6E66696775726174696F6E3A0D0A009D
:104FAE00002D2D2D2D2D2D2D2D2D2D2D2D2D2D2D50
:104FBE002D2D2D2D2D2D2D0D0A0000094D697272EE
:104FCE006F72204C6F636B75703A20446973616227
:104FDE006C65640D0A0000094D6972726F72204C87
:104FEE006F636B75702044656C61793A2000006DBB
:104FFE00730D0A00000954696D652062657477654A
:10500E00656E2063616D6572612073686F74733AAB
:10501E002000000953686F74732070657220636FEF
:10502E006C6F723A2000000D0A000009526570651F
:10503E0061742073657175656E6365200000207460
:10504E00696D652873292E0D0A000009456E61628F
:10505E006C656420436F6C6F72733A0D0A00000921
:10506E00092831292020205556203433306E6D0DFD
:10507E000A0000090928322B332920526F79616CFE
:10508E0020426C75652C2032780D0A000009092823
:10509E003229202020526F79616C20426C75652C6C
:1050AE002031780D0A0000090928332920202052CA
:1050BE006F79616C20426C75652C2031780D0A0079
:1050CE000009092834292020204379616E0D0A0039
:1050DE00000909283529202020477265656E0D0AC2
:1050EE0000000909283629202020416D6265720DC5
:1050FE000A000009092837292020205265640D0A6C
:10510E00000009092838292020204952203838303B
:10511E006E6D0D0A000009092839292020204952F8
:10512E00203934306E6D0D0A000049444C450000A4
:00000001FF
